:100000000C9485080C94C9080C94C9080C94C90870
:100010000C94C9080C94C9080C94C9080C94C9081C
:100020000C94C9080C94C9080C94C4140C9496152B
:100030000C94C9080C94C9080C94C9080C94C908FC
:100040000C94C9080C94702E0C94C9080C94C9081F
:100050000C94C9080C9468240C94C9080C94C90821
:100060000C94C9080C94C9080C94C9080C94C908CC
:100070000C94C9080C94C9080C94C9080C94C908BC
:100080000C94C9080C94C9080C94C9080C94C908AC
:100090000C94C9080C94C9080C94C9080C94C9089C
:1000A0000C94C9080C94C9080C94C90887099109D3
:1000B000A909C109090A0F0A300A150A2B0A210ADF
:1000C000260A1B0AF109D909350A03162516131742
:1000D000251613176A168D161317E216F5163C1A15
:1000E0003C1A6B1A6B1AAE1AEC1A051D051D051B7E
:1000F000051D061C061CD91C051D051DF01C01E173
:100100000137023702E10138023801E201250225F8
:1001100002E20001E10137023702E1013802380151
:10012000E10130023002E10001E10137023702E172
:100130000138023801E10107020702E1000135023E
:1001400035012002200001E10137023702E10138C8
:10015000023801E10125022502E10001E101360238
:100160003602E10138023801E10125022502E100F1
:1001700001E10136023602E10138023801E10126CF
:10018000022602E10001E10137023702E1013802F3
:100190003801E10126022602E10002E002E201301C
:1001A00002300002E002E20001E001E20002E002AF
:1001B000E3016402640002E002E30001E001E30005
:1001C00002E002E2012E022E02E10002E002E10260
:1001D000E20001E001E101E20002E001E3010602C8
:1001E0000602E30002E00001E00002E001E3011981
:1001F000021902E30002E00001E0000000F0A1F0BB
:10020000A329002B00E200E100358100001E00144C
:100210000004001D710D304D831F001A0016001BD5
:10022000000C304C002000080007000600E1042A02
:10023000002100150009001900E1084A00220017FA
:10024000000A000500000003302300E3000000E284
:1002500000000002540230E7000000E60000000445
:100260005424001C000B00110000002E7F250018F4
:10027000000D00100050004B0026000C000E003650
:100280000052002C00270012000F003700510028F8
:10029000002D001300330038714F004E0031002F45
:1002A000003474E50030810000010001000100010C
:1002B00000010000003A003500310001000100019A
:1002C000003B0035022102350001004C003C001EBD
:1002D0000224062202010001003D002D0224022416
:1002E00004010001003E000100370011040000017C
:1002F000003F00010000000100000001000E30017D
:100300000000000100000001004000240624022338
:1003100002000001004100220425023500300001E6
:100320000042002304260235023800010043002465
:100330000425041F02370001004400310026043167
:10034000023602010045001E0230022D02010000AB
:100350000001000100010001000100000001000196
:100360000001000100010001000100F400F200FBA7
:1003700000010001000100F000F100FA000100019D
:10038000000100F500F300FC00010001000100F98C
:1003900000FA00F600000001000100010000000169
:1003A0000000000100A800010000000100000001A1
:1003B0000001000100A900AA0000000100010001E5
:1003C000000100010001000100010001000100AC7A
:1003D000000100B600010001000100AB0050000167
:1003E00000010001000100520051000100AE0001B7
:1003F00000010001004F00000001000100010001A8
:1004000000010000000100010001000100010001E5
:1004100000010001000100010001000100010001D4
:1004200000010001000100010001000100010001C4
:1004300000010001000100010001000100000001B5
:100440000001000100000001000000010004300173
:1004500000000001000000010005300630093001F5
:1004600000000001000A300B3008300100010001DB
:10047000000100073001000100010001000100013E
:100480000001000100010001000100010001000164
:100490000001000100010001000100010001000055
:1004A0000001000100010001000100000001000145
:1004B00000010001000100010001000100500001E5
:1004C0000001000100010052005100010001000183
:1004D00000010001004F00010001000100010001C6
:1004E0000001000100000001000100010000000106
:1004F00000000001000100010000000100000001F7
:10050000003F00520051002302000001004000247F
:100510000021001E00270001004100250022001FCD
:1005200000370001004200260023002000270001C0
:10053000004300300230002402270201004400453D
:1005400000380001000100000001000100E100018D
:1005500000E0000000010001000100010001003D79
:100560000001000100010001000100E000010001A4
:10057000000100010001002C000100010001000148
:100580000001003C00010001000100010000003AF0
:1005900000010001000000010000003B000E3001DE
:1005A0000000000100000001000100010001000145
:1005B0000000000100010001000100010001000134
:1005C0000001000100010001000100010001000123
:1005D0000001000100010001000100010001000113
:1005E0000001000100010001000100010001000004
:1005F000000A002530313662003A2000253032589A
:10060000000A722F632030313233343536373839AF
:100610004142434445460A000A00253032580062F0
:100620006F756E6365213A20006C6566742073698E
:1006300064652061747461636865640A006C656652
:10064000742073696465206E6F7420726573706FB7
:100650006E64696E670A00747279696E6720746FE0
:10066000207265736574206D637032333031380ADF
:10067000005B735D004B6579626F61726420737417
:100680006172742E0A005B575D005B535D005B5224
:100690005D005B445D005B435D0016034500720036
:1006A00067006F0044006F007800200045005A008A
:1006B000000016034500720067006F0044006F00E1
:1006C0007800200045005A000000040309040902D4
:1006D0008D00050100A0FA090400000103010100DA
:1006E000092111010001223F000705810308000ACA
:1006F0000904010001030102000921110100012286
:100700004D000705820308000A09040200010300E6
:1007100000000921110100012236000705830308AA
:10072000000A09040300020300000009211101006E
:10073000012220000705840320000107050403208F
:100740000001090404000103000000092111010057
:100750000122390007058503100001120110010074
:10076000000008EDFE071301000102000105010968
:1007700006A101050719E029E7150025019508756F
:100780000181020508190129059505750191029558
:1007900001750391010507190029771500250195B9
:1007A0007875018102C00631FF0974A10109751530
:1007B0000025FF9520750881020976150025FF9513
:1007C0002075089102C005010980A101850216016A
:1007D0000026B7001A01002AB700751095018100A4
:1007E000C0050C0901A1018503160100269C021A0F
:1007F00001002A9C02751095018100C005010902C3
:10080000A1010901A100050919012905150025010A
:100810009505750181029501750381010501093076
:1008200009311581257F95027508810609381581E2
:10083000257F950175088106050C0A38021581256A
:100840007F950175088106C0C005010906A1010553
:100850000719E029E7150025019508750181029522
:100860000175088101050819012905950575019192
:10087000029501750391010507190029FF1500254F
:10088000FF950675088100C00A0025303258200007
:100890006B6579626F6172645F7265706F72743AD2
:1008A00020000A0025303258006B6579626F617252
:1008B000645F7365745F6C65643A200064656C5FA7
:1008C0006B65795F6269743A2063616E2774206496
:1008D000656C3A20253032580A006164645F6B65AC
:1008E000795F6269743A2063616E27742061646481
:1008F0003A20253032580A00646F6E652E0A006275
:100900006F6F676D61676963207363616E3A202E54
:100910002E2E2000290A002575002F002575005D68
:1009200028002564002000256400200025640020A4
:10093000002564007C0025303258006D6F757365AA
:100940006B6579205B62746E7C78207920762068F4
:100950005D287265702F61636C293A205B006D6BB6
:100960005F776865656C5F74696D655F746F5F6DF7
:100970006178203D2025640A006D6B5F77686565AE
:100980006C5F6D61785F7370656564203D202564E0
:100990000A006D6B5F74696D655F746F5F6D617880
:1009A000203D2025640A006D6B5F6D61785F737078
:1009B000656564203D2025640A006D6B5F696E7477
:1009C000657276616C203D2025640A006D6B5F6462
:1009D000656C6179203D2025640A006D6B5F776846
:1009E00065656C5F74696D655F746F5F6D617820BC
:1009F0003D2025640A006D6B5F776865656C5F6DEF
:100A000061785F7370656564203D2025640A006D20
:100A10006B5F74696D655F746F5F6D6178203D20F9
:100A200025640A006D6B5F6D61785F737065656446
:100A3000203D2025640A006D6B5F696E74657276D7
:100A4000616C203D2025640A006D6B5F64656C61FC
:100A500079203D2025640A000A00257500363A20D9
:100A6000776865656C5F74696D655F746F5F6D61F4
:100A7000783A20000A00257500353A2077686565C8
:100A80006C5F6D61785F73706565643A20000A0081
:100A9000257500343A2074696D655F746F5F6D6110
:100AA000783A20000A00257500333A206D61785F9E
:100AB00073706565643A20000A00257500323A209B
:100AC000696E74657276616C286D73293A20000A2C
:100AD00000257500313A2064656C6179282A31302F
:100AE0006D73293A20000A092D2056616C756573D3
:100AF000202D0A004D3E004D25643E20003F00732E
:100B000065742064656661756C740A00433E20005C
:100B100077686572652064656C74613A20637572EC
:100B2000736F723D25642C20776865656C3D256484
:100B30000A53656520687474703A2F2F656E2E779E
:100B4000696B6970656469612E6F72672F77696B75
:100B5000692F4D6F7573655F6B6579730A000A09BC
:100B60002D204D6F7573656B6579202D0A455343B4
:100B70002F713A09717569740A313A0964656C61BB
:100B800079282A31306D73290A323A09696E746501
:100B90007276616C286D73290A333A096D61785F4A
:100BA00073706565640A343A0974696D655F746FC2
:100BB0005F6D61780A353A09776865656C5F6D61CC
:100BC000785F73706565640A363A09776865656CA5
:100BD0005F74696D655F746F5F6D61780A0A703A62
:100BE000097072696E742076616C7565730A643A77
:100BF000097365742064656661756C74730A757039
:100C00003A092B310A646F776E3A092D310A706701
:100C100075703A092B31300A7067646F776E3A0944
:100C20002D31300A0A7370656564203D2064656C5F
:100C30007461202A206D61785F7370656564202A75
:100C40002028726570656174202F2074696D655F5E
:100C5000746F5F6D6178290A003F004D3E200043AC
:100C60003E20004C25640A000A092D20436F6E7354
:100C70006F6C65202D0A4553432F713A09717569D0
:100C8000740A6D3A096D6F7573656B65790A000AB0
:100C9000092D204D61676963202D0A643A09646556
:100CA0006275670A783A096465627567206D6174D8
:100CB0007269780A6B3A096465627567206B6579B9
:100CC000626F6172640A6D3A096465627567206DCE
:100CD0006F7573650A763A0976657273696F6E0A85
:100CE000733A097374617475730A633A09636F6EBA
:100CF000736F6C65206D6F64650A302D343A096C32
:100D000061796572302D34284631302D4634290AF8
:100D1000506175733A09626F6F746C6F61646572CC
:100D20000A653A09656570726F6D0A6E3A094E4B35
:100D3000524F0A7A3A09736C656570204C4544201D
:100D4000746573740A000A002575002E6E6B726F4D
:100D50003A20000A002575002E737761705F62618A
:100D6000636B736C6173685F6261636B7370616303
:100D7000653A20000A002575002E737761705F6761
:100D8000726176655F6573633A20000A002575001D
:100D90002E6E6F5F6775693A20000A002575002E78
:100DA000737761705F72616C745F726775693A2006
:100DB000000A002575002E737761705F6C616C749A
:100DC0005F6C6775693A20000A002575002E636123
:100DD00070736C6F636B5F746F5F636F6E74726F51
:100DE0006C3A20000A002575002E737761705F63EE
:100DF0006F6E74726F6C5F636170736C6F636B3A6C
:100E000020000A0025303258006B65796D61705FF3
:100E1000636F6E6669672E7261773A20000A00255B
:100E200075002E6D6F7573653A20000A00257500F8
:100E30002E6B6579626F6172643A20000A00257535
:100E4000002E6D61747269783A20000A00257500E1
:100E50002E656E61626C653A20000A0025303258BA
:100E60000064656275675F636F6E6669672E7261A5
:100E7000773A20000A0025750064656661756C7418
:100E80005F6C617965723A20003F004E4B524F3AD9
:100E9000206F66660A004E4B524F3A206F6E0A0072
:100EA00074696D65725F636F756E743A20253034B6
:100EB0006C580A006B6579626F6172645F6E6B7269
:100EC0006F3A2025580A006B6579626F6172645F22
:100ED00069646C653A2025580A006B6579626F6118
:100EE00072645F70726F746F636F6C3A2025580A7A
:100EF00000686F73745F6B6579626F6172645F6CB9
:100F000065647328293A2025580A000A092D2053C0
:100F10007461747573202D0A004743433A20342EC0
:100F2000392E33204156522D4C4942433A20312E1E
:100F3000382E31204156525F415243483A20617663
:100F400072350A004F5054494F4E533A204C554683
:100F50004120424F4F544D41474943204D4F555337
:100F6000454B45592045585452414B455920434F14
:100F70004E534F4C4520434F4D4D414E44204E4B18
:100F8000524F203531320A004255494C443A203202
:100F90003430646230632D6469727479202830398A
:100FA0003A35383A3539204A616E203238203230AD
:100FB0003136290A005649443A203078464545449E
:100FC000284572676F446F7820455A29205049445C
:100FD0003A20307831333037284572676F446F7864
:100FE00020455A29205645523A2030783030303149
:100FF0000A00444553433A20742E6D2E6B2E206B0D
:101000006579626F617264206669726D776172657D
:1010100020666F72204572676F646F780A000A0954
:101020002D2056657273696F6E202D0A000A6D6F50
:101030007573653A206F66660A000A6D6F75736591
:101040003A206F6E0A000A6B6579626F6172643ACA
:10105000206F66660A000A6B6579626F6172643A96
:10106000206F6E0A000A6D61747269783A206F66AB
:10107000660A000A6D61747269783A206F6E0A0020
:101080000A64656275673A206F6E0A000A646562D9
:1010900075673A206F66660A000A0A626F6F746CA1
:1010A0006F616465722E2E2E2000433E2000656520
:1010B000636F6E6669673A0A00536C656570204C11
:1010C000454420746573740A0000000000000000AD
:1010D00000000000010204060A0F17202C3A4A5DA6
:1010E00071879DB3C7DAE9F5FCFFFCF5E9DAC7B310
:1010F0009D87715D4A3A2C20170F0A0604020100F1
:101100000000000000000000000011241FBECFEF0F
:10111000DAE0DEBFCDBF04B603FE24C08091FB0140
:101120009091FC01A091FD01B091FE018730904BA0
:10113000A740B04BB9F41092FB011092FC01109241
:10114000FD011092FE0114BE84B7877F84BF88E141
:101150000FB6F89480936000109260000FBEE0E03C
:10116000FFE3099511E0A0E0B1E0ECE7F0E602C092
:1011700005900D92AA33B107D9F711E0AAE3B1E0C7
:1011800001C01D92AB3FB107E1F70E94FC110C9426
:101190003C300C940000FF93EF93E0913A01F09102
:1011A0003B01309709F00995EF91FF910895FC01FB
:1011B0008591803011F0EFDFFBCF0895FF27E0E24B
:1011C00030E247FF0CC0419597FF09C0EDE2609502
:1011D000709580959095611D711D811D911D27FF52
:1011E00002C0219530E350E2AA27660F771F881FBF
:1011F000991FAA1FA41710F0A41B63955A95A9F76D
:10120000AA3008F0A95FA05DAF93F3956115710551
:101210008105910541F7ED3211F4EF93F395F21743
:1012200018F43F93F395FBCF8F91B5DFFA95E1F773
:101230000895E991F9918591803021F0853219F076
:10124000AADFF9CF089520E0E89455915532C1F313
:10125000503311F4689455915A3348F4505390F335
:10126000220F022E220F220F200D250FF4CF0EF495
:10127000219589919991533619F3533729F15335B3
:1012800059F1BC0188279927E8945C3621F48991AB
:10129000999168945591543639F446EF7EF077FF72
:1012A0000DC08FEF9FEF0AC055374AE039F058352F
:1012B00040E121F0523642E009F00895FF93EF93A8
:1012C0007DDFEF91FF91B7CFFF93EF93FC01819109
:1012D0008030B9F360DFFBCFFF93EF9368DFF1CF8E
:1012E000DF93CF93CDB7DEB72596A3DFCF91DF9104
:1012F0000895462F50E04F30510508F0DEC0DC0164
:10130000FA01EA5AFF4F12968C910C94F12F882320
:1013100021F085EE0E94D918D0C085EE0E94A11957
:10132000CCC0882349F00E94322490933D018093E1
:101330003C0188EF91E0089580913C0190913D013E
:101340000E943E24873991050CF0A8C08AEE91E0F6
:101350000895882349F00E94322490933D018093A0
:101360003C0187EE91E0089580913C0190913D0110
:101370000E943E24873991050CF093C089ED91E0DD
:101380000895882349F00E94322490933D01809370
:101390003C0182ED91E0089580913C0190913D01E6
:1013A0000E943E24873991050CF07EC080EC91E0CC
:1013B0000895882349F00E94322490933D01809340
:1013C0003C018BEB91E0089580913C0190913D01AF
:1013D0000E943E24873991050CF069C08DEA91E0A6
:1013E0000895882349F00E94322490933D01809310
:1013F0003C0188EA91E0089580913C0190913D0183
:101400000E943E24873991050CF054C08AE991E08E
:101410000895882309F451C085E891E00895882350
:1014200009F44BC080E791E00895882309F445C092
:101430008BE591E00895882309F43FC086E491E0AC
:1014400008958823D1F18DE391E008958823A9F1CF
:1014500088E291E00895882381F183E191E0089585
:10146000882359F18EEF90E00895882331F180911F
:10147000BE019091BF01A091C001B091C10120E2D5
:10148000822780729927AA27BB278093BE01909359
:10149000BF01A093C001B093C1010FC085EF91E0DF
:1014A000089584EE91E008958BEC91E0089586EB29
:1014B00091E0089583EA91E0089580E090E0089536
:1014C00008956091BE017091BF018091C00190911B
:1014D000C1010E94672356985E9825982D982698FA
:1014E0002E9827982F98833099F028F4813041F076
:1014F000823049F00895843049F0853061F00895D4
:10150000259A2D9A0895269A2E9A0895259A2D9A0D
:10151000279A2F9A0895259A2D9A269A2E9A279AD5
:101520002F9A089581E69AE0892B11F00E94610AB2
:1015300080E090E0089556985E9825982D9826981A
:101540002E9827982F988FEF90E0909389008093A2
:10155000880090938B0080938A0090938D008093F5
:101560008C00259A2D9A2FEF80E792E02150804041
:101570009040E1F700C00000269A2E9A2FEF80E7F6
:1015800092E0215080409040E1F700C00000279A8F
:101590002F9A2FEF80E792E0215080409040E1F7B2
:1015A00000C0000025982D982FEF80E792E0215091
:1015B00080409040E1F700C0000026982E982FEF61
:1015C00080E792E0215080409040E1F700C00000A9
:1015D00027982F9856985E9825982D9826982E989B
:1015E00027982F98089589EA8093800089E0809356
:1015F000810024982C983F988AB18F748AB96E988C
:10160000479A8BB1806B8BB9769A0E949B0A80E6D1
:101610009AE0892B11F00E94600A80E090E0089522
:1016200080E28093000180913E0181110EC00E94F2
:101630005F0B81E080933E012FEF83ED90E321501B
:1016400080409040E1F700C0000080E40E94650BFC
:101650008093000181112EC00E948F0B80930001A6
:10166000811128C00E948F0B80930001811122C03C
:101670008FE30E948F0B8093000181111BC00E9499
:10168000870B80E40E94650B80930001811112C0DA
:101690008CE00E948F0B8093000181110BC00E948F
:1016A0008F0B80930001811105C08FE30E948F0B87
:1016B000809300010E94870B809100010895109291
:1016C000B9008AE08093B800089594EA9093BC0032
:1016D0009091BC0097FFFCCF9091B900987F983013
:1016E00021F0903111F081E008958093BB0084E8EF
:1016F0008093BC008091BC0087FFFCCF8091B90033
:10170000887F883111F0803471F780E0089584E992
:101710008093BC008091BC0084FDFCCF0895809331
:10172000BB0084E88093BC008091BC0087FFFCCFA5
:101730009091B900987F81E0983209F480E0089593
:1017400084E88093BC008091BC0087FFFCCF80912F
:10175000BB00089580910001811115C080E40E94B2
:10176000650B8093000181110CC082E10E948F0BF8
:1017700080930001811105C08FEF0E948F0B809331
:1017800000010E94870B84B1807F84B985B1807F7E
:1017900085B98AB1837F8AB98BB1837F8BB93E9833
:1017A000469808950E94100B809300010E94AA0B96
:1017B00080B38C7080BB81B3836F81BBA0E4B1E048
:1017C000EEE4F1E08EE08E0F11921D928E13FCCFAD
:1017D00083EF9AE0892B11F00C94F30A08959F92FD
:1017E000AF92BF92CF92DF92EF92FF920F931F932F
:1017F000CF93DF93809100018823E1F080913F0136
:101800008F5F80933F01811115C087E596E00E94AC
:10181000D7080E94100B80930001882329F08DE3E4
:1018200096E00E94D70806C089E296E00E94D70899
:101830000E949B0A00E411E0C0E0D0E0BB24B39416
:1018400082E0A82ECC24C394D12C2AE1E22E26E0FB
:10185000F22EC730D10500F580910001811164C0DE
:1018600080E40E94650B80930001811112C082E127
:101870000E948F0B8093000181110BC0C6010C2EBA
:1018800001C0880F0A94EAF780950E948F0B80931D
:1018900000010E94870B48C0CA30A1F028F4C8306C
:1018A00059F0C93061F005C0CC3089F070F0CD300E
:1018B00089F0209A289810C0219A29980DC0229A60
:1018C0002A980AC0239A2B9807C0529A01C0539AAB
:1018D0005B9802C03E9A469890EA9A95F1F79FB1BC
:1018E000799902C082E001C080E091709B25982B1D
:1018F0007C9902C084E001C080E0892B7D9902C000
:1019000038E001C030E0832B7E9902C020E101C0A5
:1019100020E0822B9FB19095991F9927991F92954E
:10192000990F907E892B10C080910001811174C0A5
:1019300080E40E94650B80930001882309F459C05C
:10194000912C0E94870B892DF8019081981739F10D
:10195000808380910101882301F18091D90180FF6A
:1019600004C08FE196E00E94D7088091D90180FFE2
:101970000CC0809101011F928F93FF92EF920E9401
:1019800070090F900F900F900F908091D90180FFF8
:1019900004C088E196E00E94D708A09201010E944D
:1019A000AA0B21960F5F1F4FCE30D10509F051CF02
:1019B000809101018823B1F0815080930101882337
:1019C00039F08FE99FE00197F1F700C000000AC0ED
:1019D000AEE4B1E0E0E4F1E0CF01825F91919D934C
:1019E0008E13FCCF82E99AE0892BC1F00E94920A03
:1019F00015C083E10E948F0B809300018111A0CF5D
:101A000081E40E94650B80930001811199CF0E94AF
:101A1000A00B982E909495CF80E096CF81E0DF9137
:101A2000CF911F910F91FF90EF90DF90CF90BF90DB
:101A3000AF909F900895E82FF0E0E25BFE4F808129
:101A40000895CF92DF92EF92FF920F931F93CF935F
:101A5000DF9381E096E00E94D7088EE4E82E81E0D3
:101A6000F82EC0E0D0E09CEFC92E95E0D92E03EF10
:101A700015E0DF93CF93DF92CF920E94700989EF38
:101A800095E00E94D708F70181917F0190E00E94C4
:101A9000CD239F938F931F930F930E94700981EF23
:101AA00095E00E94D70821968DB79EB708960FB68D
:101AB000F8949EBF0FBE8DBFCE30D105D1F6DF9119
:101AC000CF911F910F91FF90EF90DF90CF900895ED
:101AD0008B3B910578F4883A910540F5853A91055C
:101AE000D0F48430910508F0B1C08130910509F43B
:101AF000ADC06BC0803E910508F467C0883E91057B
:101B000008F4A4C09C01205F31092031310508F0A0
:101B10005CC090650895853A910509F459C0863AEC
:101B2000910509F058C082E890E40895883A91053B
:101B300009F454C0893A910509F453C08A3A9105D1
:101B400009F452C08B3A910509F451C08C3A9105C1
:101B500009F450C08D3A910509F44FC0803B9105BE
:101B600009F44EC08E3A910509F44DC08F3A9105A3
:101B700009F44CC0813B910509F44BC0823B9105AF
:101B800009F44AC0833B910509F449C0843B91059F
:101B900009F448C0853B910509F447C0863B91058F
:101BA00009F446C0873B910509F445C0883B91057F
:101BB00009F444C0893B910509F443C08A3B91056F
:101BC00009F442C080E094E4089580E090E0089534
:101BD00081E890E4089583E890E4089582EE94E427
:101BE000089589EE94E408958AEE94E4089585EBCF
:101BF00094E4089586EB94E4089587EB94E40895C3
:101C00008CEC94E408958DEC94E4089583E895E4D5
:101C100008958AE895E4089582E995E4089584E9B1
:101C200095E4089581E296E4089583E296E40895A8
:101C300084E296E4089585E296E4089586E296E4C7
:101C4000089587E296E408958AE296E40895089557
:101C500096E0799FF001112494E5899FE00DF11D34
:101C60001124E60FF11DEE0FFF1FEF5FFD4F859171
:101C700094910895880F991FFC01E558FF4F8591B5
:101C800094910895880F991FFC01E550FE4F8591AE
:101C90009491089526E0729FF001112444E5849FF9
:101CA000E00DF11D1124E60FF11DEE0FFF1FEF5F98
:101CB000FD4F859194919C013A9521154FE1340790
:101CC00008F41AC13F512115304120F49F700E9441
:101CD000420E08959C0130532115304118F4992784
:101CE000906C0895811520E5920769F40E94271DE4
:101CF0004FEF84E39CE0415080409040E1F700C00A
:101D000000000C948D24813020E5920731F48091FD
:101D1000D90181608093D90108959C013055211526
:101D2000304108F051C0292F33272F70332721303D
:101D30003105D9F4AC014370552702C0220F331F7F
:101D40004A95E2F73C68AC0164E0440F551F6A9580
:101D5000E1F744275370242B352B73E0880F991F2C
:101D60007A95E1F7807699271DC02230310529F454
:101D7000982F8827816F906A089523303105A9F440
:101D8000AC014370552721E030E002C0220F331F21
:101D90004A95E2F73C6843E0880F991F4A95E1F7BE
:101DA000807E9770822B932B089524303105E1F4C7
:101DB000AC014370552721E030E002C0220F331FF1
:101DC0004A95E2F73A68E7CF9C0130572115304138
:101DD00018F49F70906208959C013058211530418D
:101DE00018F49F70906A0895803E9105E0F4803C5D
:101DF000910558F58133910509F46FC048F4893293
:101E0000910509F463C08A32910509F46DC072C06E
:101E100089339105E9F082389105D1F08533910538
:101E200009F44DC067C0833E910581F138F4803ECE
:101E30009105B9F0823E9105D9F05CC0863E9105CE
:101E400061F1873E9105A1F155C00E943A0E0895B7
:101E50002091EC0120FD02C021FF4CC080EE90E0FB
:101E600049C08091EC0180FFF9CF89E390E042C046
:101E70008091EC0182FF0EC08091EC0184FF03C0D1
:101E800080E090E037C083EE90E034C08091EC01B8
:101E900082FFF2CF82EE90E02DC08091EC0183FFB3
:101EA0000BC08091EC0184FDEBCF87EE90E022C067
:101EB0008091EC0183FFF5CF86EE90E01BC080910E
:101EC000EC0185FF07C089E290E014C08091EC012D
:101ED00085FFF9CF85E390E00DC08091EC0186FF8E
:101EE00007C08AE290E006C08091EC0186FFF9CF3E
:101EF00081E390E00E94680D0895089580916F013C
:101F000008959FB7F89410925E019FBF9091F201DF
:101F1000943009F057C09091E9009F703091EC0027
:101F2000232F217030FD20E8922B24E02093E9003C
:101F30002091EB0020FF43C02091EE0027FF3FC01F
:101F400020915C01222321F02091E80025FF37C079
:101F500010925C0126E03091E80035FD15C030910B
:101F6000F201343061F53091EB0035FD28C021508D
:101F700021F481E080935C0122C0EFE9FFE031971A
:101F8000F1F700C00000E7CF8093F1008091E800F6
:101F900085FD0AC08091E80080FFFCCF8091E800B9
:101FA0008E778093E80006C08FB7F89421E02093E5
:101FB0005E018FBF9F709093E90080E008959F704D
:101FC0009093E9008FEF0895CF93DF9300D01F9295
:101FD000CDB7DEB79C018091F201843019F593E012
:101FE00099833B832A839093E9008FEF9091E800D7
:101FF000815095FD06C095ED9A95F1F7000081118D
:10200000F5CF8091E80085FF0DC040E050E063E02F
:1020100070E0CE0101960E94B4128091E8008E77A4
:102020008093E8000F900F900F90DF91CF9108956B
:10203000CF93DF9300D01F92CDB7DEB72091F2018E
:10204000243021F522E029839B838A8383E08093D7
:10205000E9008FEF9091E800815095FD06C095ED65
:102060009A95F1F700008111F5CF8091E80085FF86
:102070000DC040E050E063E070E0CE0101960E94A8
:10208000B4128091E8008E778093E8000F900F9053
:102090000F90DF91CF9108952091F2012430F1F457
:1020A00022E02093E9002FEF3091E800215035FD28
:1020B00006C035ED3A95F1F700002111F5CF2091DA
:1020C000E80025FF0BC040E050E065E070E00E94B2
:1020D000B4128091E8008E778093E8000895CF9342
:1020E000DF932091F201243009F048C0EC01809187
:1020F0000C018823E1F080910D018823C1F085E077
:102100008093E9008FEF9091E800815095FD06C023
:1021100095E19A95F1F700008111F5CF8091E800E3
:1021200085FF2CC040E050E060E170E017C081E026
:102130008093E9008FEF9091E800815095FD06C0F3
:1021400095ED9A95F1F700008111F5CF8091E800A7
:1021500085FF14C040E050E068E070E0CE010E94CE
:10216000B4128091E8008E778093E80080E1FE0150
:10217000AFE5B1E001900D928A95E1F7DF91CF9143
:10218000089586E996E00E94D7088091F1018111B7
:1021900009C00E9449140E94A6148091E200846044
:1021A0008093E200089582E996E00E94D708109299
:1021B000F10108958EE896E00C94D7088AE896E03D
:1021C0000E94D7080C945D2E86E896E00E94D708FE
:1021D0000E9423240E94632E0E944B170C947D0FB3
:1021E00020915D012F5F822F62E30E94D12F9923FE
:1021F00019F020935D01089510925D0180915E01B8
:10220000882371F18091F201843041F58091E900D9
:102210008F702091EC00922F917020FD90E8892B17
:1022200094E09093E9009091EB0090FF14C090919E
:10223000EE0097FF10C09091E80095FF03C0109248
:10224000F100F9CF9091E80090FF05C09091E8006F
:102250009E779093E8008F708093E90010925E0162
:10226000089542E061EC81E00E94C31342E061EC1A
:1022700082E00E94C31342E061EC83E00E94C3133A
:1022800042E261EC84E00E94C31342E161EC85E02C
:102290000C94C3138091F401833009F455C030F4D9
:1022A000813071F0823009F48EC008958A3009F4CB
:1022B0007AC08B3009F460C0893009F09CC020C01E
:1022C0008091F301813A09F096C08091E800877F00
:1022D0008093E8008091F7019091F801892B21F417
:1022E00060E18FE591E003C060E080E090E070E0A5
:1022F0000E94FF128091E8008B778093E800089598
:102300008091F301813209F076C08091F7019091BC
:10231000F801009719F0049709F06DC08091E8006A
:10232000877F8093E8008091E80082FD05C080915E
:10233000F2018111F8CF5FC08091F10080936F01AD
:102340008091E8008B7753C08091F301813A09F0C6
:1023500052C08091F7019091F801892B09F04BC090
:102360008091E800877F8093E8008091E80080FFFB
:10237000FCCF80910C0136C08091F3018132D9F5F8
:102380008091F7019091F801892BA9F58091E800DF
:10239000877F8093E8000E94F8138091F501809375
:1023A0000C010C94271D8091F301813221F580915D
:1023B000E800877F8093E8000E94F8138091F6017F
:1023C0008093700108958091F301813AA1F4809186
:1023D000E800877F8093E8008091E80080FFFCCFD1
:1023E000809170018093F1008091E8008E77809356
:1023F000E8000C94F813089584B7877F84BF88E1C0
:102400000FB6F89480936000109260000FBE90E0C9
:1024100080E80FB6F89480936100909361000FBE3E
:102420000E94D8170E9449140E94A6148091E200CD
:1024300084608093E20081E89FE00E9462237894A8
:102440000E942B170E94DA1782E091E00E94461743
:102450000E944B2E85E796E00E94D7088091F201FA
:10246000853089F481E796E00E94D7080E94E7232F
:102470008091F001882391F30E940F24882371F347
:102480000E949E12EBCF0E940818E8CF292F332715
:1024900023303105C9F064F42130310581F0223058
:1024A000310509F043C08DE890E02EEC36E042C0E3
:1024B00021323105F1F02232310541F137C082E19C
:1024C00090E02BE537E036C099278130910541F047
:1024D0008230910541F0892B49F5EAECF6E005C020
:1024E000E2EBF6E002C0EAE9F6E0849190E09F01B9
:1024F00021C06530D8F4E62FF0E0EE0FFF1FEB5D52
:10250000FE4F2081318189E090E014C0653070F485
:1025100070E0FB01EE0FFF1FE55EFE4F2081318171
:10252000FB01EA5EFE4F808190E004C080E090E015
:1025300020E030E0FA0131832083089580E189BDF5
:1025400082E189BD09B400FEFDCF8091D8008F7D66
:102550008093D8008091E00082608093E0008091B9
:10256000E00081FDFCCF0895CF92DF92EF92FF92C1
:102570000F931F93CF93DF93EC018B016A010E94AD
:102580001714811133C0C114D10439F0F6018081D0
:102590009181081B190BC80FD91FE12CF12C0115D3
:1025A000110519F18091E80085FD16C08091E800C1
:1025B0008E778093E800C114D10449F0F601808140
:1025C0009181E80EF91EF182E08285E00FC00E9441
:1025D0001714882321F30AC089918093F1000150D8
:1025E0001109FFEFEF1AFF0ADACF80E0DF91CF91F8
:1025F0001F910F91FF90EF90DF90CF900895209161
:10260000F9013091FA012617370748F06115710575
:1026100039F42091E8002E772093E80001C0B90139
:1026200040E061157105A9F12091F201222309F41E
:1026300043C0253009F442C02091E80023FD40C08A
:102640002091E80022FD32C02091E80020FFE9CF70
:102650004091F3002091F20030E0342BFC01CF01D7
:102660006115710559F02830310540F4819180934E
:10267000F100615071092F5F3F4FF1CF41E02830E9
:10268000310509F040E02091E8002E772093E80022
:10269000C8CF4111C9CF0AC08091F201882361F0EF
:1026A000853061F08091E80083FD0AC08091E800E8
:1026B00082FFF2CF80E0089582E0089583E00895DC
:1026C00081E008952091F9013091FA01261737072A
:1026D00048F06115710539F42091E8002E772093B8
:1026E000E80001C0B901FC0120E06115710591F11C
:1026F0008091F201882309F440C0853009F43FC07D
:102700008091E80083FD3DC08091E80082FD2FC0EC
:102710008091E80080FFE9CF2091F3008091F200E2
:1027200090E0922B6115710559F08830910540F4C5
:1027300024912093F1003196615071090196F2CFF6
:1027400021E0089709F020E08091E8008E778093DF
:10275000E800CBCF2111CCCF0AC08091F2018823B1
:1027600061F0853061F08091E80083FD0AC08091BE
:10277000E80082FFF2CF80E0089582E0089583E0D0
:10278000089581E00895982F973058F59093E900C7
:10279000981739F07091EC002091ED005091F00005
:1027A00003C0242F762F50E021FF19C03091EB0099
:1027B0003E7F3093EB003091ED003D7F3093ED0094
:1027C0003091EB0031603093EB007093EC0020937C
:1027D000ED005093F0002091EE0027FF07C09F5FAF
:1027E000D3CF8F708093E90081E0089580E0089551
:1027F0008091F30187FF11C08091E80082FD05C040
:102800008091F2018111F8CF11C08091E8008B779F
:102810000BC08091F201882349F08091E80080FF8D
:10282000F8CF8091E8008E778093E800089520919A
:10283000E4003091E50095E64091EC00842F817032
:1028400040FF22C08091E80080FD1CC08091F20111
:10285000882391F0853091F08091EB0085FD10C0C8
:102860004091E4005091E5004217530729F39A0183
:10287000915011F784E0089582E0089583E008956F
:1028800081E0089580E008954091E80042FFDECFA6
:1028900008950E94B7140E94BF14E0EEF0E080811A
:1028A00081608083E8EDF0E080818F77808319BCC0
:1028B000A7EDB0E08C918E7F8C9380818F7E80839A
:1028C0001092F10108950F931F93CF93DF930E940D
:1028D000B7140E94BF14C8EDD0E088818F77888339
:1028E00088818068888388818F7D888319BC109255
:1028F000F2011092EE011092F0011092EF0100EE41
:1029000010E0F80180818B7F8083888181608883DB
:1029100042E060E080E00E94C313E1EEF0E08081DD
:102920008E7F8083E2EEF0E0808181608083808111
:1029300088608083F80180818E7F808388818061B8
:102940008883DF91CF911F910F910895E8EDF0E01A
:1029500080818F7E8083E7EDF0E0808181608083DD
:1029600084E082BF81E08093F1010C946314E8ED70
:10297000F0E080818E7F80831092E20008951092B3
:10298000DA001092E10008951F920F920FB60F9295
:1029900011242F933F934F935F936F937F938F9364
:1029A0009F93AF93BF93EF93FF938091E10082FFDA
:1029B0000BC08091E20082FF07C08091E1008B7F15
:1029C0008093E1000E94F0108091DA0080FF1FC028
:1029D0008091D80080FF1BC08091DA008E7F8093A9
:1029E000DA008091D90080FF0DC080E189BD82E1CD
:1029F00089BD09B400FEFDCF81E08093F2010E9401
:102A0000C11005C019BC1092F2010E94D310809130
:102A1000E10080FF19C08091E20080FF15C0809125
:102A2000E2008E7F8093E2008091E20080618093DB
:102A3000E2008091D80080628093D80019BC85E0C4
:102A40008093F2010E94DE108091E10084FF30C08B
:102A50008091E20084FF2CC080E189BD82E189BDC4
:102A600009B400FEFDCF8091D8008F7D8093D800FF
:102A70008091E1008F7E8093E1008091E2008F7E63
:102A80008093E2008091E20081608093E200809177
:102A9000EE01882311F084E007C08091E30087FDF8
:102AA00002C081E001C083E08093F2010E94E41043
:102AB0008091E10083FF29C08091E20083FF25C05F
:102AC0008091E100877F8093E10082E08093F201B2
:102AD0001092EE018091E1008E7F8093E100809161
:102AE000E2008E7F8093E2008091E200806180931B
:102AF000E20042E060E080E00E94C3138091F000B9
:102B000088608093F0000E94DA10FF91EF91BF91EE
:102B1000AF919F918F917F916F915F914F913F9175
:102B20002F910F900FBE0F901F9018951F920F922C
:102B30000FB60F9211242F933F934F935F936F9390
:102B40007F938F939F93AF93BF93CF93DF93EF9335
:102B5000FF93C091E900CF708091EC00D82FD17025
:102B600080FDD0E81092E9008091F000877F80938B
:102B7000F00078940E94DA151092E9008091F0003C
:102B800088608093F000CD2BCF70C093E900FF9157
:102B9000EF91DF91CF91BF91AF919F918F917F91F5
:102BA0006F915F914F913F912F910F900FBE0F90BA
:102BB0001F9018951F93CF93DF93CDB7DEB7AA97D9
:102BC0000FB6F894DEBF0FBECDBFE3EFF1E088E0B3
:102BD0008E0F9091F10091938E13FBCF0E944A11BA
:102BE0008091E80083FF1FC18091F3019091F4016F
:102BF000492F50E04A30510508F015C1FA01EB5950
:102C0000FF4F0C94F12F803881F0823809F00BC10E
:102C10008091F7018F708093E9008091EB0085FB34
:102C2000882780F91092E90006C08091EF01909109
:102C3000F001911182609091E800977F9093E800F5
:102C40008093F1001092F100C8C0282F2D7F09F069
:102C5000EAC0882319F0823061F0E5C08091F50167
:102C6000813009F0E0C0933009F080E08093F001FA
:102C70002BC08091F501811127C08091F7018F70E1
:102C800009F4D1C08093E9002091EB0020FF1CC023
:102C9000933021F48091EB00806214C09091EB009E
:102CA00090619093EB0021E030E0A90102C0440F55
:102CB000551F8A95E2F74093EA001092EA0080914E
:102CC000EB0088608093EB001092E9008091E800AF
:102CD000877F86C08111A7C01091F5011F77809171
:102CE000E3008078812B8093E3008091E800877F68
:102CF0008093E8000E94F8138091E80080FFFCCFE9
:102D00008091E30080688093E300111102C082E0AB
:102D100001C083E08093F20186C08058823008F0C1
:102D200082C08091F5019091F6018C3D53E09507AA
:102D300079F583E08A838AE289834FB7F894DE01CC
:102D4000139620E03EE051E2E32FF0E0509357006D
:102D5000E49120FF03C0E295EF703F5FEF708E2F8C
:102D600090E0EA3010F0C79601C0C0968D939D9315
:102D70002F5F243149F74FBF8091E800877F809310
:102D8000E8006AE270E0CE0101960E94FF1214C0D2
:102D9000AE014F5F5F4F6091F7010E944612BC0188
:102DA000892B09F440C09091E800977F9093E80048
:102DB00089819A810E9462138091E8008B778093C9
:102DC000E80031C0803879F58091E800877F8093F2
:102DD000E8008091EE018093F1008091E8008E7709
:102DE0008093E8000E94F8131EC081111CC09091CE
:102DF000F5019230C0F48091E800877F8093E8006D
:102E00009093EE010E94F8138091EE01811106C0AB
:102E10008091E30087FD02C081E001C084E08093DF
:102E2000F2010E9431118091E80083FF0AC0809175
:102E3000E800877F8093E8008091EB0080628093B8
:102E4000EB00AA960FB6F894DEBF0FBECDBFDF91A0
:102E5000CF911F910895CF938091F2018823A1F023
:102E6000C091E900CF709091EC00892F817090FDA6
:102E700080E8C82B1092E9008091E80083FD0E9451
:102E8000DA15CF70C093E900CF9108959093760141
:102E9000809375010895E0917501F0917601309766
:102EA00021F00190F081E02D099480E00895EF92E7
:102EB000FF920F931F93CF93DF93E0917501F091F1
:102EC00076013097B1F18C010280F381E02D0995F4
:102ED0008091D90182FF2DC080FF04C080E998E075
:102EE0000E94D708E80110E18AE8E82E88E0F82E71
:102EF0008091D90180FF0BC088811F928F93FF9230
:102F0000EF920E9470090F900F900F900F90115048
:102F100021961111EDCF8091D90180FF0AC088E878
:102F200098E0DF91CF911F910F91FF90EF900C945B
:102F3000D708DF91CF911F910F91FF90EF900895E7
:102F4000E0917501F0917601309721F00480F581D0
:102F5000E02D099408952091730130917401821736
:102F6000930771F09093740180937301E091750160
:102F7000F0917601309721F00680F781E02D0994D9
:102F8000089520917101309172018217930771F0B9
:102F90009093720180937101E0917501F091760137
:102FA000309721F00084F185E02D0994089508956B
:102FB0000C94D7170E9429240E94D20B0C94EF2462
:102FC000CF93C82F8091D90182FF1EC080FF04C01B
:102FD00089EA98E00E94D7088091D90180FF0CC04F
:102FE0001F92CF9384EA98E09F938F930E94700979
:102FF0000F900F900F900F908091D90180FF04C027
:1030000082EA98E00E94D7088C2FCF910C947D0F14
:10301000CF92DF92EF92FF920F931F93CF93DF93A4
:10302000CDB7DEB72B970FB6F894DEBF0FBECDBF7E
:103030000E94EF0B88E7C82E81E0D82E00E010E058
:10304000E02E802F0E941B0DF60141916F01F42E9E
:10305000F826B1F40F5F1F4F0E30110589F78FEF7F
:1030600089838A831B820E9432248160782F9D830A
:103070008C8349815A816B818D810E94AB1840C03D
:103080009091D90191FF04C08B870E94210D8B85FF
:1030900020E030E04F2D50E0922FBA01022E02C006
:1030A000759567950A94E2F760FF24C02E83EF823E
:1030B00021E030E0690102C0CC0CDD1C9A95E2F7FA
:1030C00090E08C219D21892B09F420E028870E9423
:1030D00032248160782F9A8789874E815F81688545
:1030E0008A850E94AB18F801E858FE4F8081C826F7
:1030F000C08206C02F5F3F4F2630310569F6AACF48
:103100000E946028109177010E944B171817A1F0B8
:103110000E944B17809377012B960FB6F894DEBF71
:103120000FBECDBFDF91CF911F910F91FF90EF9018
:10313000DF90CF900C94E0172B960FB6F894DEBF7B
:103140000FBECDBFDF91CF911F910F91FF90EF90F8
:10315000DF90CF900895CF93DF93CDB7DEB72B9755
:103160000FB6F894DEBF0FBECDBF4F835887698777
:103170007A878B87DE01119686E0FD0111928A9590
:10318000E9F785E0FE01379601900D928A95E1F707
:1031900049815A816B817C818D819E810E94C11FF2
:1031A0002B960FB6F894DEBF0FBECDBFDF91CF9147
:1031B0000895CF93882309F4C2C0C82F823859F4E8
:1031C0000E944B1781FDBBC089E30E945D220E94D3
:1031D0003C2389E30CC0833879F40E944B1780FDAF
:1031E000AEC083E50E945D220E943C2383E50E94DD
:1031F000B022CF910C943C23843859F40E944B1791
:1032000082FD9DC087E40E945D220E943C2387E4EA
:10321000EECF8CEF8C0F813A48F48C2F0E94F32C68
:1032200081118DC08C2F0E945D22E3CF80E28C0F34
:10323000883048F4C77081E001C0880FCA95EAF76A
:103240000E940523D6CF8BE58C0F833078F4C53AE6
:1032500029F0C63A31F083E890E005C081E890E0BB
:1032600002C082E890E0CF910C94AB1788E58C0FF8
:10327000833108F064C0C83A39F1C93A41F1CA3A19
:1032800049F1CB3A51F1CC3A59F1CD3A61F1C03B19
:1032900069F1CE3A71F1CF3A79F1C13B81F1C23B8C
:1032A00089F1C33B91F1C43B99F1C53BA1F1C63B08
:1032B000A9F1C73BB1F1C83BB9F1C93BC1F1CA3B68
:1032C000C9F180E090E038C082EE90E035C089EE30
:1032D00090E032C08AEE90E02FC085EB90E02CC0E9
:1032E00086EB90E029C087EB90E026C08CEC90E064
:1032F00023C08DEC90E020C083E891E01DC08AE8F7
:1033000091E01AC082E991E017C084E991E014C00D
:1033100081E292E011C083E292E00EC084E292E08A
:103320000BC085E292E008C086E292E005C087E229
:1033300092E002C08AE292E0CF910C94C117CF9143
:103340000895882309F44BC0823859F40E944B1722
:1033500081FF45C089E30E945D220E943C2389E3EE
:103360000CC0833871F40E944B1780FF38C083E58E
:103370000E945D220E943C2383E50E94B0220C94AF
:103380003C23843859F40E944B1782FF28C087E4FD
:103390000E945D220E943C2387E4EFCF9CEF980FB0
:1033A000913A58F390E2980F983050F4877091E07A
:1033B00001C0990F8A95EAF7892F0E940B23DFCF6E
:1033C0009BE5980F933020F480E090E00C94AB17CD
:1033D000885A833120F480E090E00C94C11708955E
:1033E000882321F00E9405230C943C230895882310
:1033F00021F00E940B230C943C230895BF92CF929E
:10340000DF92EF92FF920F931F93CF93DF9300D041
:1034100000D000D0CDB7DEB725E0FC01DE0111966B
:1034200001900D922A95E1F7FC01408131810281E2
:10343000258122952F7063817481672B09F4E5C281
:103440003F3F19F44F3F09F4E0C27C0149833A83BE
:1034500089819A812E830E941C22182FB92E0E94E6
:103460001B220E94E220EB2DE295EF70F0E0E15983
:10347000FF4F2E810C94F12F8B2D807F9B2D9F7001
:10348000F92E882319F0F29480EFF822002349F0F6
:10349000FF2009F467C28F2D0E9415230E943C2350
:1034A00061C2812F0E94A119FF2009F4AEC28F2DA5
:1034B0000E941B2326960FB6F894DEBF0FBECDBF29
:1034C000DF91CF911F910F91FF90EF90DF90CF9000
:1034D000BF900C943C233B2D307F8B2D8F7030326E
:1034E00011F08295807F112319F0113021F12CC049
:1034F0000023B9F0222309F4A0C1213009F09DC1B5
:1035000026960FB6F894DEBF0FBECDBFDF91CF91E8
:103510001F910F91FF90EF90DF90CF90BF900C9490
:103520002523222319F0213009F46FC28E830E94D3
:1035300028238E8196C1002321F0223008F065C235
:103540007CC1211162C28DC1002321F0222309F424
:1035500074C108C2222309F484C119C22B2D2695F7
:103560002695237030E02115310521F021303105F9
:10357000D1F04BC2002321F0812F9B2D937002C00C
:1035800080E090E026960FB6F894DEBF0FBECDBF68
:10359000DF91CF911F910F91FF90EF90DF90CF902F
:1035A000BF900C94AB17002321F0812F9B2D9370BB
:1035B00002C080E090E026960FB6F894DEBF0FBE02
:1035C000CDBFDF91CF911F910F91FF90EF90DF90D2
:1035D000CF90BF900C94C117812F002319F00E9447
:1035E000E62602C00E944E2726960FB6F894DEBF4C
:1035F0000FBECDBFDF91CF911F910F91FF90EF9044
:10360000DF90CF90BF900C94D3278B2D837009F05F
:103610007BC00111FAC1812F829586958770880F32
:10362000880F912F9F70C92ED12CE12CF12C082EE0
:1036300004C0CC0CDD1CEE1CFF1C0A94D2F714FF56
:1036400012C04FE050E060E070E004C0440F551F2E
:10365000661F771F8A95D2F7CB01BA0160957095E6
:103660008095909503C060E070E0CB012B2D2695EE
:1036700026952370422F50E042305105D9F0433057
:10368000510569F16C297D298E299F294130510509
:1036900051F126960FB6F894DEBF0FBECDBFDF9175
:1036A000CF911F910F91FF90EF90DF90CF90BF903F
:1036B0000C9409216C297D298E299F2926960FB605
:1036C000F894DEBF0FBECDBFDF91CF911F910F9158
:1036D000FF90EF90DF90CF90BF900C9425210E9437
:1036E0000921C701B60126960FB6F894DEBF0FBEBA
:1036F000CDBFDF91CF911F910F91FF90EF90DF90A1
:10370000CF90BF900C94ED20002319F08B2D817089
:1037100001C08695882309F478C1812F829586950A
:103720008770880F880F912F9F70C92ED12CE12CA4
:10373000F12C082E04C0CC0CDD1CEE1CFF1C0A94DE
:10374000D2F714FF12C04FE050E060E070E004C018
:10375000440F551F661F771F8A95D2F7CB01BA0118
:10376000609570958095909503C060E070E0CB0106
:103770002B2D269526952370422F50E0423051057F
:10378000D9F04330510569F16C297D298E299F2993
:103790004130510551F126960FB6F894DEBF0FBEA9
:1037A000CDBFDF91CF911F910F91FF90EF90DF90F0
:1037B000CF90BF900C94E3216C297D298E299F29FD
:1037C00026960FB6F894DEBF0FBECDBFDF91CF9126
:1037D0001F910F91FF90EF90DF90CF90BF900C94CE
:1037E000FF210E94E321C701B60126960FB6F89487
:1037F000DEBF0FBECDBFDF91CF911F910F91FF9024
:10380000EF90DF90CF90BF900C94C721103FD1F183
:1038100018F4103E50F4A1C0123F09F463C008F43C
:103820004CC0133F09F473C098C01F708B2D8F716B
:103830000023A1F00E946021812F26960FB6F894F4
:10384000DEBF0FBECDBFDF91CF911F910F91FF90D3
:10385000EF90DF90CF90BF900C94F0190E948121DF
:10386000812F26960FB6F894DEBF0FBECDBFDF9135
:10387000CF911F910F91FF90EF90DF90CF90BF906D
:103880000C94F7190023A9F02111BFC08B2D8F7163
:1038900026960FB6F894DEBF0FBECDBFDF91CF9155
:1038A0001F910F91FF90EF90DF90CF90BF900C94FD
:1038B000A621223008F0A9C0E9CF0023A9F08B2D62
:1038C0008F7126960FB6F894DEBF0FBECDBFDF9185
:1038D000CF911F910F91FF90EF90DF90CF90BF900D
:1038E0000C946021002359F38B2D8F7126960FB60F
:1038F000F894DEBF0FBECDBFDF91CF911F910F9126
:10390000FF90EF90DF90CF90BF900C948121002327
:1039100099F08B2D8F7126960FB6F894DEBF0FBEEF
:10392000CDBFDF91CF911F910F91FF90EF90DF906E
:10393000CF90BF900C944B2126960FB6F894DEBF23
:103940000FBECDBFDF91CF911F910F91FF90EF90F0
:10395000DF90CF90BF900C9441210023A9F0222347
:1039600009F4ADCF812F26960FB6F894DEBF0FBEB7
:10397000CDBFDF91CF911F910F91FF90EF90DF901E
:10398000CF90BF900C94D918222309F4ADCF812F8A
:1039900026960FB6F894DEBF0FBECDBFDF91CF9154
:1039A0001F910F91FF90EF90DF90CF90BF900C94FC
:1039B000A1194B2D4F70612FC7010E9479092696DE
:1039C0000FB6F894DEBF0FBECDBFDF91CF911F9130
:1039D0000F91FF90EF90DF90CF90BF900C946520F7
:1039E0004B2D4F70612FC70126960FB6F894DEBF9E
:1039F0000FBECDBFDF91CF911F910F91FF90EF9040
:103A0000DF90CF90BF900C94270E26960FB6F894B7
:103A1000DEBF0FBECDBFDF91CF911F910F91FF9001
:103A2000EF90DF90CF90BF9008950E9422230E94D4
:103A3000F7220E943C230E9406290E94D32780E09F
:103A400090E00E94AB1780E090E00C94C1170E94B8
:103A500012230C94151D0E941C22292F22952F70D1
:103A600030E02C3031054CF42A3031056CF4225012
:103A700031092230310588F407C02C30310549F076
:103A80002F30310531F009C0803E48F0803F29F4E5
:103A900006C093FB882780F9089580E0089581E0AF
:103AA0000895CF93DF9300D000D01F92CDB7DEB73B
:103AB0000F900F900F900F900F90DF91CF9108957E
:103AC000CF93DF9300D000D000D0CDB7DEB72696DD
:103AD0000FB6F894DEBF0FBECDBFDF91CF91089532
:103AE0001F93CF93DF93C091860116E080918701E9
:103AF000C81799F0D0E01C9FF0011D9FF00D112414
:103B0000E857FE4F408151816281738184819581A4
:103B10000E94601D2196C770E9CFDF91CF911F9160
:103B200008954091B8015091B9016091BA01709126
:103B3000BB018091BC019091BD010C94601D8091EE
:103B4000BD0182958F7009F054C08091BA0188231D
:103B500009F44FC080918601A09187016091B8015E
:103B60007091B9014091BB015091BC01B6E08A1738
:103B700009F43FC090E041155105C1F17F3F11F4B8
:103B80006F3FA1F1B89FF001B99FF00D1124E857E4
:103B9000FE4F218172132AC02081621327C0228127
:103BA000211124C0238134812417350710F42150BA
:103BB0003109241B350B283C3105C0F42091BD018F
:103BC0002F7020612093BD0126E0289FF001299FDE
:103BD000F00D1124E357FE4F80818F708061808348
:103BE00088EB91E00E94FE190C94701D019687707D
:103BF000BECF0895CF92DF92EF92FF920F931F9363
:103C0000CF93DF93CDB7DEB762970FB6F894DEBFE0
:103C10000FBECDBF8C0185E0F801DE011D9601903D
:103C20000D928A95E1F7D8014C9111965C9111970C
:103C300012966C9112971396CD90DC901497309158
:103C4000B8017091B9018091BB019091BC010097BE
:103C500009F46BC17F3F19F43F3F09F466C1E0905E
:103C6000BA01EE2009F4C0C02091BD01C816D906E2
:103C700028F0F601E81BF90BCF0104C08095909560
:103C80008C0D9D1DFF24F394883C910578F0F12C58
:103C9000207F09F0C6C07C2DD98AC88A89890E94F4
:103CA000511D88EB91E00E94FE19B1C0822F807FE8
:103CB00009F046C0751314C0341312C0611110C04E
:103CC0002F7020612093BD010E94911D88EB91E02F
:103CD0000E94FE198091BD01D80115968C932EC0CB
:103CE000CD2819F15F3F11F44F3FF9F0F62E611125
:103CF0001CC0809186012091870136E0821709F46B
:103D00005AC090E0389FF001399FF00D1124E85718
:103D1000FE4F7181571306C07081471303C0728133
:103D2000711103C001968770E9CFF62E662309F45E
:103D300018C18091BD0181608093BD01F12C11C13A
:103D4000751308C0341306C0611104C08091BD0111
:103D5000D801C3C04D875E878D859E856A8B0E9482
:103D60002B1D6A898823E1F16623D1F12091BD01E1
:103D7000822F82958F7090E0029774F08091B80145
:103D80009091B90198878F831986DB86CA862C8724
:103D9000CE0107960E94FE1986E0F801A8EBB1E07B
:103DA00001900D928A95E1F70E949F1D0E94911D3E
:103DB000FF24F394D6C04D875E878D859E850E9433
:103DC0001C22292F22952F7030E0223031050CF073
:103DD000BCC09F7009F0B6C0805E883008F4C1C0D6
:103DE000C8010E94FE19E4CFC816D90608F453C0D2
:103DF000F601E81BF90BCF01883C910508F450C08F
:103E0000F12C7C2DD98AC88A89890E94511DE8EB42
:103E1000F1E086E0DF011D928A95E9F70E94911D8D
:103E2000A0C0751314C0341312C0611110C080916A
:103E3000BD01F8018583C8010E94FE1986E0E8EB08
:103E4000F1E0DF011D928A95E9F7FE2C8AC04D87CB
:103E50005E878D859E856A8B0E942B1D6A898823CB
:103E600009F4BECF662309F4BBCF2091BD01822F98
:103E700082958F7090E002970CF48ECF8091B801FC
:103E80009091B9019A8389831B82DD82CC822E8333
:103E9000CE0101967FCF809590958C0D9D1DACCF66
:103EA000F62E662309F49CCF75132EC034132CC054
:103EB0002091BD0120FD1FC0822F82958F70D9F007
:103EC000D80115962C9315978F3049F08F5F982F56
:103ED0009295907F822F8F70892B15968C93C801B5
:103EE0000E94FE1986E0F801A8EBB1E001900D9266
:103EF0008A95E1F793CF86E0F801A8EBB1E0019055
:103F00000D928A95E1F72DC04D875E878D859E8540
:103F10000E942B1D811140CF8091BD018160809353
:103F2000BD01C8010E94FE191CC0662309F458CFC8
:103F30004D875E878D859E850E942B1D882309F401
:103F40004FCF2ACF811148CF0CC0243031050CF05F
:103F500047CF9F7009F440CFF8019581907F09F019
:103F60003BCF8F2D62960FB6F894DEBF0FBECDBF4C
:103F7000DF91CF911F910F91FF90EF90DF90CF9045
:103F800008951F93CF93DF93CDB7DEB72C970FB66D
:103F9000F894DEBF0FBECDBF4F83588769877A87FD
:103FA0008B879C87CE0107960E94FA1D882369F0B3
:103FB0008F8198852A853B85232BF1F19F3F09F05E
:103FC00063C08F3F09F060C037C086E0FE013796BE
:103FD000DE01119601900D928A95E1F76F81788547
:103FE000EA85FB85309741F17F3F11F46F3F21F166
:103FF0002091870130E0C90101968770992740918F
:10400000860150E08417950709F447C069837A83D5
:10401000FD83EC8396E0929FD001939FB00D112415
:10402000A857BE4FFE01319601900D929A95E1F787
:10403000809387010E94701D16E080918601909107
:1040400087018917C1F1189FC001112488579E4F1D
:104050000E94FA1D882379F1E09186011E9FF001EC
:104060001124E857FE4F4081518162817381848120
:1040700095810E94601D8091860190E00196877075
:10408000992780938601D9CF4F81588569857A8594
:104090008B859C850E94601DCFCF0E94271D1092AA
:1040A000870110928601E8EBF1E086E0DF011D92C6
:1040B0008A95E9F7C1CF2C960FB6F894DEBF0FBEF4
:1040C000CDBFDF91CF911F910895EF92FF920F9393
:1040D0001F93CF93DF938C01892B09F46CC0F12CD3
:1040E000EE24E394E8012196F8018491843740F4AA
:1040F000843008F051C0813081F0823019F15BC00A
:10410000853709F444C0A8F19CE7980F903708F070
:1041100052C08F770E94A11941C00E5F1F4FFE0150
:10412000C49180E28C0F883048F4C7708E2D01C096
:10413000880FCA95EAF70E94152314C08C2F0E949D
:10414000D9182DC00E5F1F4FFE01C49180E28C0F65
:10415000883058F4C7708E2D01C0880FCA95EAF7D1
:104160000E941B230E943C231AC08C2F0E94A1197D
:1041700016C00E5F1F4FFE01C491CC2381F08FE962
:104180009FE00197F1F700C00000C150F6CF0E5F2D
:104190001F4FFE01F49003C00E94D9188E018F2D8D
:1041A000882309F49FCFEFE9FFE03197F1F700C0D2
:1041B00000008150F5CFDF91CF911F910F91FF90BB
:1041C000EF90089508956093C2017093C3018093A6
:1041D000C4019093C5010C94151D0F931F9300917A
:1041E000C2011091C3012091C4013091C501DC01CD
:1041F000CB01802B912BA22BB32B8093C2019093E8
:10420000C301A093C401B093C5011F910F910C94F9
:10421000151D0F931F930091C2011091C3012091AE
:10422000C4013091C501DC01CB0180239123A2237D
:10423000B3238093C2019093C301A093C401B093B0
:10424000C5011F910F910C94151D0F931F930091A1
:10425000C2011091C3012091C4013091C501DC015C
:10426000CB0180279127A227B3278093C201909387
:10427000C301A093C401B093C5011F910F910C9489
:10428000151D1092BE011092BF011092C001109234
:10429000C1010C94151D41E050E060E070E004C0E5
:1042A000440F551F661F771F8A95D2F74093BE01B2
:1042B0005093BF016093C0017093C1010C94151D10
:1042C00041E050E060E070E004C0440F551F661FFD
:1042D000771F8A95D2F78091BE019091BF01A0917E
:1042E000C001B091C101482B592B6A2B7B2B409305
:1042F000BE015093BF016093C0017093C1010C9443
:10430000151D41E050E060E070E004C0440F551F0F
:10431000661F771F8A95D2F74095509560957095E6
:104320008091BE019091BF01A091C001B091C101E7
:10433000482359236A237B234093BE015093BF0136
:104340006093C0017093C1010C94151D41E050E0D1
:1043500060E070E004C0440F551F661F771F8A9508
:10436000D2F78091BE019091BF01A091C001B091A0
:10437000C101482759276A277B274093BE015093E4
:10438000BF016093C0017093C1010C94151D0F9380
:104390001F930091BE011091BF012091C001309187
:1043A000C101DC01CB01802B912BA22BB32B80937D
:1043B000BE019093BF01A093C001B093C1011F91B2
:1043C0000F910C94151D0F931F930091BE01109136
:1043D000BF012091C0013091C101DC01CB018023DC
:1043E0009123A223B3238093BE019093BF01A09396
:1043F000C001B093C1011F910F910C94151D0F9333
:104400001F930091BE011091BF012091C001309116
:10441000C101DC01CB0180279127A227B32780931C
:10442000BE019093BF01A093C001B093C1011F9141
:104430000F910C94151D0895CF92DF92EF92FF9289
:104440000F931F93CF93DF938C01C090C201D09044
:10445000C301E090C401F090C5014091BE015091AC
:10446000BF016091C0017091C101C42AD52AE62A1A
:10447000F72ACFE1D0E0D701C6010C2E04C0B695D3
:10448000A795979587950A94D2F780FF07C0B80142
:104490008C2F0E944A0E8130910531F4219758F7F4
:1044A000B80180E00E944A0EDF91CF911F910F91D9
:1044B000FF90EF90DF90CF90089590910C01992399
:1044C00021F090910D01911109C020910E013091C0
:1044D0000F01F90132969FEF40E030C0982F96957A
:1044E000969596959F30A0F4E0910E01F0910F0102
:1044F000E90FF11D877021E030E0A90102C0440FEF
:10450000551F8A95E2F7CA019181892B818308950D
:104510009091D90190FF23C01F928F938AED98E06C
:104520009F938F930E9470090F900F900F900F90A0
:1045300008959F3F39F04F5F4E3041F0519158132D
:10454000F8CF0DC05111F7CF942FF5CF9F3F39F021
:10455000F901E90FF11D97FDFA95828308950895F9
:1045600090910C01992321F090910D01911109C0B6
:1045700020910E0130910F01F9013296205F3F4FDB
:1045800030C0982F9695969596959F30A8F4E09117
:104590000E01F0910F01E90FF11D877021E030E06D
:1045A000A90102C0440F551F8A95E2F7CA01809500
:1045B00091818923818308959091D90190FF16C03C
:1045C0001F928F938CEB98E09F938F930E947009BA
:1045D0000F900F900F900F9008953196E217F30708
:1045E00029F090819813F9CF1082F7CF089581E0D8
:1045F00090E0E0910E01F0910F01E80FF91F108299
:10460000019680319105A9F708959091D801892BE1
:104610008093D801089580959091D8018923809343
:10462000D80108951092D80108959091D701892B4F
:104630008093D701089580959091D7018923809325
:10464000D70108951092D70108958093C601089567
:104650001092C601089580910E0190910F01FC0106
:1046600031969C01205F3F4F80E0919191118F5FC7
:10467000E217F307D1F70895E0910E01F0910F01D1
:104680008091D8018083E0910E01F0910F0190811B
:104690008091D701892B80838091C601882361F0A6
:1046A000E0910E01F0910F019081892B80830E948F
:1046B0002B2381111092C60180910E0190910F0160
:1046C0000C94571790933B0180933A010895CF9231
:1046D000DF92EF92FF926C01EE24FF24C114D1040B
:1046E000E104F10421F0C701B60120E101C020E09E
:1046F000C72ED82EE92EFF24C114D104E104F10401
:1047000019F0285FC701B6016B017C0154E0F694F3
:10471000E794D794C7945A95D1F7C114D104E10412
:10472000F10419F02C5FC701B6016B017C0142E076
:10473000F694E794D794C7944A95D1F7C114D1045D
:10474000E104F10419F02E5FC701B601DC01CB01D1
:10475000B695A79597958795892B8A2B8B2B09F072
:104760002F5F822FFF90EF90DF90CF90089582957A
:10477000982F9C7C392F36953695282F237344E04B
:10478000249FC0011124932F982B292F2A7A269534
:10479000892F8575880F822B08951F93CF93DF9300
:1047A0001F92CDB7DEB799830E94B723182F998146
:1047B000892F0E94B723212F30E0322F2227A90111
:1047C000482BCA010F90DF91CF911F9108958091DE
:1047D000F201843009F11092DA0120E488E190E0DE
:1047E0000FB6F894A895809360000FBE20936000E8
:1047F00083B7817F846083BF83B7816083BF7894F0
:10480000889583B78E7F83BF88E10FB6F894809335
:104810006000109260000FBE089508950895CF9330
:104820000E940D240E94EF0B0E940E24C0E08C2FEA
:104830000E941B0D811104C0CF5FCE30C1F701C0B3
:1048400081E0CF9108950E94271D0E944B170C9480
:104850007D0F82E084BD93E095BD9AEF97BD809374
:104860006E0008952FB7F8948091DB019091DC01E0
:10487000A091DD01B091DE012FBF0895CF92DF92AC
:10488000EF92FF920F931F932FB7F8944091DB01A3
:104890005091DC016091DD017091DE012FBF6A0152
:1048A0007B01EE24FF248C0120E030E0C016D1060D
:1048B000E206F30610F4415051099A01281B390B06
:1048C000C9011F910F91FF90EF90DF90CF90089555
:1048D0001F920F920FB60F9211248F939F93AF9355
:1048E000BF938091DB019091DC01A091DD01B0913B
:1048F000DE010196A11DB11D8093DB019093DC01C7
:10490000A093DD01B093DE01BF91AF919F918F9194
:104910000F900FBE0F901F9018950E944914F894A5
:104920002FEF87EA91E6215080409040E1F700C0E8
:10493000000087E090EBDC018093FB019093FC0189
:10494000A093FD01B093FE019CE088E10FB6F894BE
:10495000A895809360000FBE90936000FFCFEF9208
:10496000FF920F931F93CF93DF93D82FC0E08C2F2C
:104970000E941B0D00E010E0E82EF12CC701002E74
:1049800002C0959587950A94E2F780FD06C00F5FF7
:104990001F4F0630110591F709C0602F7C2F80E072
:1049A0000E94280ED813F3CF81E004C0CF5FCE3031
:1049B000F1F680E0DF91CF911F910F91FF90EF9082
:1049C0000895CF93C82F8CE20E94AF24882321F052
:1049D0008C2FCF910C94AF2480E0CF910895CF938A
:1049E0000E943E26811102C00E9424268FEF98E08B
:1049F0000E94D708C5E6C15049F00E94EF0B8FE333
:104A00009CE90197F1F700C00000F5CF88EF98E02E
:104A10000E94D70889E20E94E124811113C18AE231
:104A20000E94E12481110E94242685E00E94E12455
:104A300081110E948D240E9449268093D90187E02C
:104A40000E94E1248823A9F18BE10E94E1248823BC
:104A500051F08091D90181FB222720F991E0922722
:104A600090FB81F90EC08EE00E94E124882361F062
:104A70008091D90182FB222720F991E0922790FBB7
:104A800082F98093D90115C080E10E94E1249091C0
:104A9000D901882341F093FB222720F981E0822766
:104AA00080FB93F904C0892F809580FB90F9909347
:104AB000D9018091D9010E944D260E945B268093E6
:104AC000EC0180EE0E94E124882341F08091EC010A
:104AD000982F909590FB80F98093EC0189E30E94D8
:104AE000E124882359F08091EC0181FB222720F9F1
:104AF00091E0922790FB81F98093EC0182EE0E9475
:104B0000E124882359F08091EC0182FB222720F9CF
:104B100091E0922790FB82F98093EC0186EE0E944F
:104B2000E124882359F08091EC0183FB222720F9AE
:104B300091E0922790FB83F98093EC0183EE0E9431
:104B4000E124882359F08091EC0184FB222720F98D
:104B500091E0922790FB84F98093EC0185E30E9419
:104B6000E124882359F08091EC0185FB222720F96C
:104B700091E0922790FB85F98093EC0181E30E94FC
:104B8000E124882359F08091EC0186FB222720F94B
:104B900091E0922790FB86F98093EC0181E10E94DD
:104BA000E124882359F08091EC0187FB222720F92A
:104BB00091E0922790FB87F98093EC018091EC01C2
:104BC0000E945F268091EC0187FB882780F9809303
:104BD0000D0187E20E94E124C82F8EE10E94E124AA
:104BE0008111C2608FE10E94E1248111C46080E2E2
:104BF0000E94E1248111C86081E20E94E1248111B8
:104C0000C06182E20E94E1248111C06283E20E94BD
:104C1000E1248111C06484E20E94E124882311F020
:104C2000C06802C0CC2329F08C2F0E9456266C2F1E
:104C300003C00E945226682F70E080E090E0CF9180
:104C40000C94E320CF9108956DEE7EEF80E090E02C
:104C50000E94273060E082E090E00E94193060E01E
:104C600083E090E00E94193060E084E090E00E94D0
:104C7000193060E085E090E00C94193080E090E01D
:104C80000E94133021E08D3E9E4F09F020E0822FDC
:104C9000089582E090E00C940B30682F82E090E061
:104CA0000C94193083E090E00C940B30682F83E073
:104CB00090E00C94193084E090E00C940B30682F55
:104CC00084E090E00C9419308091E10180FF0BC0EA
:104CD0006091130185E0689FB00111247595679577
:104CE000759567952BC081FF09C06091130185E020
:104CF000689FB00111247595679520C082FF07C099
:104D00006091130185E0689FB001112417C0909154
:104D1000E2019923D1F060911201961788F7209152
:104D2000130185E0289F90011124929FA001939F79
:104D3000500D112470E0CA010E94DD2F603871050A
:104D400040F46115710539F002C065E070E0862F0E
:104D500008958FE7089581E008958091E10180FF33
:104D600008C06091110170E075956795759567951C
:104D700021C081FF06C06091110170E075956795B3
:104D800019C082FF04C06091110170E010C09091C1
:104D9000E2019923C1F0609110019617A0F780916C
:104DA0001101899FC001112470E00E94DD2F60383D
:104DB000710528F46115710521F0862F08958FE79C
:104DC000089581E0089561E070E0F4CF803F21F420
:104DD0000E946426819504C0813F29F40E946426C4
:104DE0008093E5010895823F21F40E946426819515
:104DF00004C0833F29F40E9464268093E40108954F
:104E0000893F19F40E94AD2605C08A3F31F40E9403
:104E1000AD2681958093E60108958B3F21F40E9491
:104E2000AD26819504C08C3F29F40E94AD26809365
:104E3000E7010895843F21F48091E301816017C068
:104E4000853F21F48091E301826011C0863F21F407
:104E50008091E30184600BC0873F21F48091E301DE
:104E6000886005C0883F31F48091E30180618093C0
:104E7000E30108958D3F21F48091E10181600BC031
:104E80008E3F21F48091E101826005C08F3F29F4BB
:104E90008091E10184608093E1010895803F39F4BD
:104EA0008091E50187FF6CC01092E50169C0813FE8
:104EB00029F48091E5011816BCF362C09091E401D9
:104EC000823F29F497FF5CC01092E40159C0833FF0
:104ED00019F41916CCF354C0893F41F48091E601CE
:104EE00018160CF04DC01092E6014AC08A3F29F412
:104EF0008091E60187FF44C0F6CF8B3F39F4809163
:104F0000E70187FF3DC01092E7013AC08C3F29F4CA
:104F10008091E7011816BCF333C0843F21F48091DF
:104F2000E3018E7F17C0853F21F48091E3018D7FDF
:104F300011C0863F21F48091E3018B7F0BC0873F36
:104F400021F48091E301877F05C0883F31F480918F
:104F5000E3018F7E8093E30113C08D3F21F48091A4
:104F6000E1018E7F0BC08E3F21F48091E1018D7FA6
:104F700005C08F3F29F48091E1018B7F8093E1018F
:104F80008091E40181110EC08091E50181110AC078
:104F90008091E601811106C08091E701811102C074
:104FA0001092E20108958091D90183FF7EC08BE3C6
:104FB00099E00E94D7088091E3011F928F9386E3C6
:104FC00099E09F938F930E94700984E399E00E9477
:104FD000D7088091E401282F332727FD30953F9390
:104FE0008F9381E399E09F938F930E9470098FE2E2
:104FF00099E00E94D7088091E501282F332727FDEB
:1050000030953F938F938CE299E09F938F930E940A
:1050100070098AE299E00E94D7088091E601282F62
:10502000332727FD30953F938F9387E299E09F9335
:105030008F930E94700985E299E00E94D7088091C1
:10504000E701282F332727FD30953F938F9382E286
:1050500099E09F938F930E9470098FE199E00E94DD
:10506000D7088091E2011F928F938CE199E09F9382
:105070008F930E9470098AE199E00E94D70880917D
:10508000E1011F928F9387E199E09F938F930E9494
:10509000700984E199E00E94D7088DB79EB74C96BD
:1050A0000FB6F8949EBF0FBE8DBF83EE91E00E94B5
:1050B000A0170E9432249093E0018093DF010895AD
:1050C0001F93CF93DF938091DF019091E0010E94C5
:1050D0003E24AC019091E201992321F0209114012A
:1050E00030E006C0209115018AE0289F900111242C
:1050F0004217530708F486C08091E401C091E5018E
:10510000D091E6011091E701811107C0C11176C06D
:10511000D11174C0111172C075C09F3F19F09F5F0B
:105120009093E201181624F40E9464268093E4010F
:105130008091E40187FF05C00E94642681958093D9
:10514000E4011C1624F40E9464268093E5018091FA
:10515000E50187FF05C00E94642681958093E501E3
:105160006091E401662339F1C091E501CC2319F186
:10517000772767FD7095872F972F0E94E22E23E3F4
:1051800033E343E35FE30E94462F0E94AF2E609318
:10519000E4016C2F772767FD7095872F972F0E946A
:1051A000E22E23E333E343E35FE30E94462F0E94B2
:1051B000AF2E6093E5011D1624F40E94AD26809366
:1051C000E6018091E60187FF05C00E94AD2681952A
:1051D0008093E601111624F40E94AD268093E70126
:1051E0008091E70187FF05C00E94AD2681958093DD
:1051F000E701DF91CF911F910C94D3279F3F09F0D6
:105200008ECF96CFDF91CF911F910895E3EEF1E01D
:1052100085E0DF011D928A95E9F71092E201109274
:10522000E10108958EE59BE00E94D7081F9281E07E
:105230008F931F9285E08F9380E19BE09F938F93E4
:105240000E9470090F900F900F900F900F900F9089
:1052500008958330E9F128F4813061F0823009F15A
:105260000895853009F462C008F449C0863009F415
:1052700074C0089580911501262F30E0280F311D4C
:105280002F3F310524F4680F6093150103C08FEFA1
:1052900080931501809115011F928F9389E49AE004
:1052A00072C080911401262F30E0280F311D2F3F4E
:1052B000310524F4680F6093140103C08FEF8093CD
:1052C0001401809114011F928F9387E39AE05BC0D1
:1052D00080911301262F30E0280F311D2F3F31051B
:1052E00024F4680F6093130103C08FEF80931301C0
:1052F000809113011F928F9384E29AE044C08091C1
:105300001201262F30E0280F311D2F3F310524F4E4
:10531000680F6093120103C08FEF80931201809198
:1053200012011F928F938FE09AE02DC0809111019E
:10533000262F30E0280F311D2F3F310524F4680F50
:105340006093110103C08FEF8093110180911101CF
:105350001F928F9386EF99E016C080911001262F3F
:1053600030E0280F311D2F3F310524F4680F609382
:10537000100103C08FEF80931001809110011F92E4
:105380008F938BED99E09F938F930E9470090F90FC
:105390000F900F900F900895833081F128F48130A1
:1053A00059F08230D1F00895853009F449C0B8F140
:1053B000863009F456C0089580911501681720F4CD
:1053C000861B8093150102C0109215018091150172
:1053D0001F928F938CEC99E054C080911401681750
:1053E00020F4861B8093140102C010921401809156
:1053F00014011F928F938AEB99E043C080911301AF
:10540000681720F4861B8093130102C010921301C9
:10541000809113011F928F9387EA99E032C08091A7
:105420001201681720F4861B8093120102C01092AB
:105430001201809112011F928F9382E999E021C09D
:1054400080911101681720F4861B8093110102C01E
:1054500010921101809111011F928F9389E799E0B9
:1054600010C080911001681720F4861B80931001F2
:1054700002C010921001809110011F928F938EE54F
:1054800099E09F938F930E9470090F900F900F9057
:105490000F900895CF93C82F1F928F9383E69CE0BF
:1054A0009F938F930E94700981E090E0A0E0B0E0AC
:1054B000BC01CD0104C0660F771F881F991FCA95D4
:1054C000D2F70E94E3200F900F900F900F90CF9192
:1054D0000C94271DCF938D3109F465C0B0F58E3043
:1054E00009F4CCC100F5873009F49BC1A8F48630DB
:1054F00009F06DC28091D901817F8E7F8093D9019F
:1055000088E69CE00E94D7088AEA90E10E94D708CA
:1055100081E08093E90180C1883009F44FC08B306D
:1055200009F47CC154C2863109F4F0C138F48031E9
:1055300009F4B8C1813109F430C249C2893109F492
:10554000CEC18B3109F486C142C2853309F437C21A
:1055500048F4873209F433C208F433C2893209F4BB
:105560002EC235C2833438F48A3308F02CC2883313
:1055700009F454C12CC2833409F421C2883409F0DF
:1055800026C20E94271D89E990E10E94D7089FEF5B
:1055900023ED80E3915020408040E1F700C00000FF
:1055A0000E948D2439C189EB90E10E94D7080E94A6
:1055B000692E0E944B170E947D0F2EC18EEA90E14A
:1055C0000E94D70889E79EE00E94D7080E945226D1
:1055D0001F928F9386E79EE09F938F930E9470099E
:1055E00084E79EE00E94D7080E944926C82F81E6E2
:1055F0009EE00E94D7081F92CF938CE59EE09F9378
:105600008F930E9470098AE59EE00E94D70880E58A
:105610009EE00E94D7088C2F81701F928F938DE49B
:105620009EE09F938F930E9470098BE49EE00E94FE
:10563000D70881E49EE00E94D708C1FB882780F943
:105640001F928F938EE39EE09F938F930E94700929
:105650008CE39EE00E94D70880E39EE00E94D7087A
:10566000C2FB882780F91F928F938DE29EE09F9363
:105670008F930E9470098BE29EE00E94D70882E21D
:105680009EE00E94D708C3FBCC27C0F91F92CF939E
:105690008FE19EE09F938F930E9470098DE19EE0C1
:1056A0000E94D7080E945B26C82F89E09EE00E94D6
:1056B000D7081F92CF9384E09EE09F938F930E9420
:1056C000700982E09EE00E94D70889EE9DE00E946A
:1056D000D7088C2F81701F928F9386EE9DE09F9349
:1056E0008F930E9470098DB79EB780960FB6F8947D
:1056F0009EBF0FBE8DBF84EE9DE00E94D7088DEC4B
:105700009DE00E94D708C1FB882780F91F928F93E4
:105710008AEC9DE09F938F930E94700988EC9DE036
:105720000E94D70886EB9DE00E94D708C2FB88271D
:1057300080F91F928F9383EB9DE09F938F930E943C
:10574000700981EB9DE00E94D7088FE99DE00E94DF
:10575000D708C3FB882780F91F928F938CE99DE0BF
:105760009F938F930E9470098AE99DE00E94D70859
:1057700080E99DE00E94D708C4FB882780F91F922A
:105780008F938DE89DE09F938F930E9470098BE823
:105790009DE00E94D70889E79DE00E94D708C5FBDD
:1057A000882780F91F928F9386E79DE09F938F93C0
:1057B0000E94700984E79DE00E94D70888E59DE07B
:1057C0000E94D708C6FB882780F91F928F9385E532
:1057D0009DE09F938F930E94700983E59DE00E9456
:1057E000D7088BE49DE00E94D708C7FBCC27C0F9FF
:1057F0001F92CF9388E49DE09F938F930E9470093E
:1058000086E49DE00E94D7088DB79EB74C960FB6F0
:10581000F8949EBF0FBE8DBFC1E0DEC08FE89CE054
:105820005BC08091D901C82FC17080FF09C08CE88E
:1058300090E10E94D7088091D901817F8E7F47C077
:1058400080E890E10E94D7088091D901816080931F
:10585000D901E2CF9091D90191FBCC27C0F981E029
:10586000C827892FC0FB81F98093D901CC2319F077
:1058700083E790E127C085E690E12EC09091D901A1
:1058800092FBCC27C0F981E0C827892FC0FB82F9A1
:105890008093D901CC2319F086E590E113C086E40A
:1058A00090E11AC09091D90193FBCC27C0F981E017
:1058B000C827892FC0FB83F98093D901CC2351F0ED
:1058C0008AE390E10E94D7088091D901816080939A
:1058D000D90182C08DE290E10E94D7089DCF8EE170
:1058E00090E10E94D70882EF9FE00E94D70885EBE5
:1058F0009FE00E94D70888E89FE00E94D70884E4D0
:105900009FE00E94D70889E19FE0E6CF8BE09FE00F
:105910000E94D7080E944B171F928F9381EF9EE041
:105920009F938F930E94700980910C011F928F9317
:105930008AED9EE09F938F930E9470098091700181
:105940001F928F9387EC9EE09F938F930E94700924
:1059500080910D011F928F9384EB9EE09F938F9314
:105960000E9470098091DB019091DC01A091DD0122
:10597000B091DE01BF93AF939F938F9380EA9EE037
:105980009F938F930E9470098DB79EB746960FB66E
:10599000F8949EBF0FBE8DBF3FCF0E94271DC091C0
:1059A0000D0181E0C827C0930D01CC2329F086E9C1
:1059B0009EE00E94D70810C08BE89EE08DCF80E06B
:1059C00003C08D5101C089530E944A2A25CF89E81E
:1059D0009EE00E94D708C0E08C2FCF91089580E010
:1059E000089580E00895CF93C82F8091E901813018
:1059F00081F020F0823009F44FC045C1E0910E01E2
:105A0000F0910F018081813169F0823209F03DC14E
:105A100009C0E0910E01F0910F018081813111F0F8
:105A2000823261F48C2F0E94EF2C811104C08C2FE4
:105A30000E946A2A2FC081E090E02CC08C2F0E9427
:105A4000F12C811126C0C431E1F070F4CB3081F02B
:105A5000C031D1F40E9412298BE59CE00E94D70846
:105A600082E08093E90115C0C93259F0C83361F46E
:105A700088E69CE00E94D7088FE59CE00E94D7084A
:105A800008C01092E90103C189E59CE00E94D70893
:105A9000FEC081E08170FDC0C43220F5CE3108F037
:105AA000C0C0CB3099F1C8F4C73009F0D2C08AE049
:105AB0008093150194E19093140193E09093130166
:105AC0008093120188E08093110188E28093100195
:105AD0008FEF9AE00E94D708BFC0C33149F1C431AB
:105AE000C1F0B7C0CB3409F4A9C028F4C93289F099
:105AF000C83361F0AEC0C13509F49EC0C23509F4A7
:105B000099C0CE3409F0A5C06AE09EC00E94122957
:105B1000A3C08091E801882319F01092E8019CC08D
:105B20008CE09BE00E94D70881E08093E901B1C03E
:105B300086EE9AE00E94D70884ED9AE00E94D7088A
:105B4000809115011F928F9381ED9AE09F938F931F
:105B50000E9470098FEC9AE00E94D7088DEB9AE0C2
:105B60000E94D708809114011F928F938AEB9AE0CC
:105B70009F938F930E94700988EB9AE00E94D70848
:105B800089EA9AE00E94D708809113011F928F93AF
:105B900086EA9AE09F938F930E94700984EA9AE0C4
:105BA0000E94D70883E99AE00E94D70880911201E9
:105BB0001F928F9380E99AE09F938F930E947009C0
:105BC0008EE89AE00E94D70889E79AE00E94D708F9
:105BD000809111011F928F9386E79AE09F938F9394
:105BE0000E94700984E79AE00E94D7088DE59AE048
:105BF0000E94D708809110011F928F938AE59AE046
:105C00009F938F930E94700988E59AE00E94D708BD
:105C10008DB79EB748960FB6F8949EBF0FBE8DBF46
:105C20001BC0CE51EC2FF0E0E15DFE4F80818093F0
:105C3000E80112C061E003C061E006C06AE0809143
:105C4000E8010E94292908C08091E8010E94CC291E
:105C500003C08DEF9AE013C08091E801882369F0BA
:105C60001F928F9387EF9AE09F938F930E94700902
:105C70000F900F900F900F9004C084EF9AE00E9455
:105C8000D70881E006C01092E90180E002C080E000
:105C900001CFCF910895E1E8F0E0808188608083B2
:105CA0008081816080838FB7F89493E0909389001E
:105CB00090ED909388008FBF0895EFE6F0E080812B
:105CC000826080830895EFE6F0E080818D7F80839D
:105CD0000895EFE6F0E0908182E0892780830895BF
:105CE0001F920F920FB60F9211242F933F934F9351
:105CF0005F936F937F938F939F93AF93BF93EF9334
:105D0000FF938091EA019091EB0101969093EB0152
:105D10008093EA01811103C082E00E947D0FE0912F
:105D2000EB01E695E695F0E0E753FF4EE4918091B4
:105D3000EA018E1303C080E00E947D0FFF91EF9176
:105D4000BF91AF919F918F917F916F915F914F9193
:105D50003F912F910F900FBE0F901F90189504D078
:105D60006894B1118DC0089570D088F09F5790F05D
:105D7000B92F9927B751A0F0D1F0660F771F881F70
:105D8000991F1AF0BA95C9F712C0B13081F077D0D7
:105D9000B1E0089574C0672F782F8827B85F39F075
:105DA000B93FCCF3869577956795B395D9F73EF4CF
:105DB00090958095709561957F4F8F4F9F4F089577
:105DC000E89409C097FB3EF4909580957095619595
:105DD0007F4F8F4F9F4F9923A9F0F92F96E9BB274B
:105DE0009395F695879577956795B795F111F8CFC7
:105DF000FAF4BB0F11F460FF1BC06F5F7F4F8F4F32
:105E00009F4F16C0882311F096E911C0772321F027
:105E10009EE8872F762F05C0662371F096E8862FBF
:105E200070E060E02AF09A95660F771F881FDAF716
:105E3000880F9695879597F9089557FD9058440FC8
:105E4000551F59F05F3F71F04795880F97FB991FD9
:105E500061F09F3F79F08795089512161306140696
:105E6000551FF2CF4695F1DF08C016161706180623
:105E7000991FF1CF86957105610508940895E894FE
:105E8000BB2766277727CB0197F908950BD078C0F9
:105E900069D028F06ED018F0952309F05AC05FC081
:105EA0001124EECFCADFA0F3959FD1F3950F50E0F8
:105EB000551F629FF001729FBB27F00DB11D639FBC
:105EC000AA27F00DB11DAA1F649F6627B00DA11D62
:105ED000661F829F2227B00DA11D621F739FB00D08
:105EE000A11D621F839FA00D611D221F749F332778
:105EF000A00D611D231F849F600D211D822F762F11
:105F00006A2F11249F5750408AF0E1F088234AF00D
:105F1000EE0FFF1FBB1F661F771F881F9150504059
:105F2000A9F79E3F510570F014C0AACF5F3FECF374
:105F3000983EDCF3869577956795B795F795E79545
:105F40009F5FC1F7FE2B880F911D9695879597F956
:105F5000089597F99F6780E870E060E008959FEFEB
:105F600080EC089500240A941616170618060906F0
:105F7000089500240A9412161306140605060895BF
:105F8000092E0394000C11F4882352F0BB0F40F447
:105F9000BF2B11F460FF04C06F5F7F4F8F4F9F4F87
:105FA0000895991B79E004C0991F961708F0961B75
:105FB000881F7A95C9F78095089597FB072E16F4E8
:105FC000009407D077FD09D00E94F72F07FC05D079
:105FD0003EF4909581959F4F0895709561957F4F00
:105FE0000895EE0FFF1F0590F491E02D0994AA1B70
:105FF000BB1B51E107C0AA1FBB1FA617B70710F0B4
:10600000A61BB70B881F991F5A95A9F780959095E5
:10601000BC01CD010895F999FECF92BD81BDF89ADA
:10602000992780B50895A8E1B0E042E050E00C94D3
:106030002E30262FF999FECF1FBA92BD81BD20BD0B
:106040000FB6F894FA9AF99A0FBE019608950E9435
:106050001930272F0C941A30DC01CB01FC01F9997F
:10606000FECF06C0F2BDE1BDF89A319600B40D92A4
:0C60700041505040B8F70895F894FFCF5D
:10607C0020027E0F6F104C101810E40F0101C701A5
:10608C0028080A03140A3F4D3620394908FC07C674
:10609C0007A6076D07E006F90612072B074B070149
:0A60AC0002030405060708090000BE
:00000001FF
